:100000000428FF3FFF3FFF3F0130031383129F008F
:100010000E3083169F00013085008601870188011C
:100020008901831285018601870188018901A00168
:10003000A101A201A301A401A501A601A701A80194
:100040000130A9002A088600013088001F150230FF
:10005000FB00FF30FA00FB0B2E283128FA0B2E286C
:100060002B284A30FA00FA0B332883161E08831215
:10007000B2070208B2072B088600023088001F155D
:100080000230FB00FF30FA00FB0B47284A28FA0B2E
:10009000472844284A30FA00FA0B4C2883161E08D9
:1000A0008312B3070208B3072C08860004308800C7
:1000B0001F150230FB00FF30FA00FB0B602863289D
:1000C000FA0B60285D284A30FA00FA0B652883167F
:1000D0001E088312B4070208B4072D0886000830F2
:1000E00088001F150230FB00FF30FA00FB0B792857
:1000F0007C28FA0B792876284A30FA00FA0B7E28F9
:1001000083161E088312B5070208B5072E0886005D
:10011000103088001F150230FB00FF30FA00FB0B87
:1001200092289528FA0B92288F284A30FA00FA0B69
:10013000972883161E088312B6070208B6072F08F1
:100140008600203088001F150230FB00FF30FA00C7
:10015000FB0BAB28AE28FA0BAB28A8284A30FA00D4
:10016000FA0BB02883161E088312B7070208B707D8
:1001700030088600403088001F150230FB00FF3039
:10018000FA00FB0BC428C728FA0BC428C1284A3040
:10019000FA00FA0BC92883161E088312B807020852
:1001A000B80731088600803088001F150230FB0038
:1001B000FF30FA00FB0BDD28E028FA0BDD28DA28F7
:1001C0004A30FA00FA0BE22883161E088312B90798
:1001D0000208B907A80A28081F3A031DFE292908A2
:1001E000200203181029AA0D2A100730F400320843
:1001F000F00000227808F0007008BA007008003A99
:10020000031D10292A142A08013A031D102903305E
:10021000F4003308F00000227808F0007008A00015
:100220002908210203183129AB0D2B100730F400E7
:100230003308F00000227808F0007008BA00700857
:10024000003A031D31292B142B08013A031D3129D3
:100250000330F4003408F00000227808F000700841
:10026000A1002908220203185229AC0D2C100730D6
:10027000F4003408F00000227808F0007008BA009A
:100280007008003A031D52292C142C08013A031D52
:1002900052290330F4003508F00000227808F000FD
:1002A0007008A2002908230203187329AD0D2D1030
:1002B0000730F4003508F00000227808F0007008DC
:1002C000BA007008003A031D73292D142D08013A55
:1002D000031D73290330F4003608F000002278086B
:1002E000F0007008A3002908240203189429AE0D19
:1002F0002E100730F4003608F00000227808F000D5
:100300007008BA007008003A031D94292E142E08B4
:10031000013A031D94290330F4003708F00000224D
:100320007808F0007008A400290825020318B529F0
:10033000AF0D2F100730F4003708F00000227808C6
:10034000F0007008BA007008003A031DB5292F1498
:100350002F08013A031DB5290330F4003808F000D6
:1003600000227808F0007008A5002908260203186A
:10037000D629B00D30100730F4003808F000002204
:100380007808F0007008BA007008003A031DD629FA
:1003900030143008013A031DD6290330F40039081F
:1003A000F00000227808F0007008A6002908270253
:1003B0000318F729B10D31100730F4003908F000A7
:1003C00000227808F0007008BA007008003A031D97
:1003D000F72931143108013A031DF7290330F400DD
:1003E0003208F00000227808F0007008A700A90A7F
:1003F0002908043A031DFD29A901A8012228FF2983
:1004000003138312F8010830FC00700DF80D740816
:10041000F80203180D2AF8070310F00DFC0B052A4B
:100420000800FF3FFF3FFF3FFF3FFF3FFF3FFF3F12
:02400E003A3F37
:00000001FF
